:100000000C9468000C9490000C9490000C94900058
:100010000C9490000C9490000C9490000C94900020
:100020000C9490000C9490000C9490000C94900010
:100030000C9490000C9490000C9490000C94900000
:100040000C9459070C9490000C9490000C94900020
:100050000C9490000C9490000C9490000C949000E0
:100060000C9487040C949000000000090003020027
:10007000000405080000000000000000000000016E
:10008000020408102040800102040810200102042C
:100090000810204080400404040404040404020204
:1000A000020202020303030303030202030000002F
:1000B0000023002600290000000000250028002B56
:1000C0000000000000240027002A0000BC021304E6
:1000D00011241FBECFEFD8E0DEBFCDBF11E0A0E0FE
:1000E000B1E0E6E4F5E102C005900D92A232B1075D
:1000F000D9F723E0A2E2B1E001C01D92AE3AB20707
:10010000E1F710E0C8E6D0E004C02197FE010E94AC
:100110009B0AC636D107C9F70E945A090C94A10A56
:100120000C940000CF93DF9369E082EE92E00E948E
:10013000060461E085E00E94C60861E089E00E9453
:10014000C60861E08AE00E94C608C3E0D1E062E030
:1001500089910E94C60881E0C830D807C1F770E0D5
:1001600060E085E00E94400870E060E089E00E9465
:10017000400870E060E08AE00E9440081092CD02E2
:100180001092CE021092CF021092D0021092D102A1
:100190001092DB021092DC021092DD021092DE025D
:1001A0001092DF021092E0021092E102DF91CF91F3
:1001B00008950F931F93CF93DF938B01EA01BC0146
:1001C00085E00E944008B80189E00E944008BE0115
:1001D0008AE0DF91CF911F910F910C94400850E07D
:1001E00040E070E060E090E080E00C94D900823064
:1001F000A9F028F4882341F0813041F0089583303C
:10020000A1F08430B9F008950C94EF0050E040E084
:1002100070E060E08FEF90E00C94D90050E040E097
:100220006FEF70E090E080E0F7CF4FEF50E070E0CC
:1002300060E0F8CF4FE750E06FE770E08FE790E0C5
:10024000EBCFFF920F931F93CF93DF931092020196
:1002500002E211E0D0E0C0E0FC2E6EE1C8010E9495
:10026000CA066093D2027093D3028093D402909313
:10027000D50260327340810591050CF47CC0E09199
:10028000DA02EE2351F0F0E0E652FD4F2081CE017C
:1002900001962817190609F46EC083E00E94F70042
:1002A0008091DA02E82FF0E0E552FD4FF394F082FE
:1002B0008F5F8093DA020E94A3076093D602709347
:1002C000D7028093D8029093D9021092010168E579
:1002D00072E080E090E00E94D4070E94EF008091DD
:1002E000DA02873001F590910201ABEDB2E0E8E06F
:1002F000F1E080E03D912191321709F444C0109261
:10030000020180910201813009F047C082E00E9421
:10031000F70060E777E180E090E00E94D407109258
:1003200002010E94EF008091DA02873009F03FC09D
:100330008091DA02873059F084E00E94F70068E586
:1003400072E080E090E00E94D4070E94EF001092DB
:10035000DB021092DC021092DD021092DE0210929B
:10036000DF021092E0021092E10281E0809301012D
:100370001092DA0234C02196025E1F4FC730D105B9
:1003800009F06ACFACCF863009F491E08F5F8730F7
:1003900009F0B0CF90930201B4CF81E00E94F70042
:1003A00068EB7BE080E090E00E94D407BACF0E9427
:1003B000A3070091D6021091D7022091D802309164
:1003C000D902601B710B820B930B60317742810560
:1003D000910528F080910101882309F4A9CFDF91CC
:1003E000CF911F910F91FF9008950F931F93CF937B
:1003F0001092C70203E011E0C0E0F80181918F0183
:100400000E9430098093C602CF5F81117EC0E091C7
:10041000CC02EE2359F0F0E0E453FD4F2081C801F7
:10042000835091402817190609F46FC083E00E9499
:10043000F70068E572E080E090E00E94D4070E9437
:10044000EF008091CC02E82FF0E0E353FD4FC08332
:100450008F5F8093CC020E94A3076093C8027093C1
:10046000C9028093CA029093CB021092000180913E
:10047000CC02853039F58091CD02813081F49091A4
:10048000CE02923061F49091CF02933041F490917A
:10049000D002943021F49091D1029530D1F1109294
:1004A000C7028091C7028130B9F582E00E94F7004F
:1004B00060E777E180E090E00E94D4071092C702E5
:1004C0000E94EF008091CC02853081F58091CC02B2
:1004D000853059F084E00E94F70068E572E080E022
:1004E00090E00E94D4070E94EF001092CD0210927B
:1004F000CE021092CF021092D0021092D10281E06F
:10050000809300011092CC0229C0C53009F075CF4C
:10051000AECF8093C702C5CF81E00E94F70068EBA1
:100520007BE080E090E00E94D407CACF0E94A3073E
:100530000091C8021091C9022091CA023091CB02E9
:10054000601B710B820B930B603177428105910523
:1005500028F080910001882309F4B8CFCF911F9132
:100560000F91089566E273E082EE92E00E940E041D
:100570000E9421010C94F50140E16FE088EA92E0CD
:100580000E94A70541E16FE08AE892E00E94A7057A
:1005900040E06FE08CE692E00E94A70541E06FE04A
:1005A0008EE492E00E94A70542E06FE080E392E0D3
:1005B0000E94A70543E06FE082E192E00E94A70558
:1005C00044E06FE084EF91E00E94A7058EE1E8EA45
:1005D000F2E0A2E2B1E001900D928A95E1F78EE19E
:1005E000EAE8F2E0A0E4B1E001900D928A95E1F72B
:1005F0008EE1ECE6F2E0AEE5B1E001900D928A9575
:10060000E1F78EE1EEE4F2E0ACE7B1E001900D92AB
:100610008A95E1F78EE1E0E3F2E0AAE9B1E001902A
:100620000D928A95E1F78EE1E2E1F2E0A8EBB1E00C
:1006300001900D928A95E1F78EE1E4EFF1E0A6EDED
:10064000B1E001900D928A95E1F708958091020141
:1006500061E0813031F08091C70262E0813009F0C1
:1006600060E082EE92E00C94980390E080E00895C0
:100670008091150390911603891B990B0895909111
:100680001603809115032FEF3FEF981748F4E92FD9
:10069000F0E0E95EFC4F208130E09F5F909316030D
:1006A000C9010895E091160380911503E81730F40D
:1006B000F0E0E95EFC4F808190E008958FEF9FEFBE
:1006C00008950895CF93DF93EC01E091EE02F0914D
:1006D000EF023097F1F0909116038091150398176F
:1006E000C0F090E0292F30E02617370754F4DE01E0
:1006F000A20FB31F4C91295E3C4FD9014C939F5FD1
:10070000F1CF1092160360931503CB01DF91CF91C7
:100710000994DF91CF910895E091F002F091F102F8
:10072000309729F01092F4021092F3020994089580
:10073000CF93DF931F92CDB7DEB769832091F2028A
:100740002223F9F02091F302203258F021E030E02A
:10075000FC013383228390E080E00F90DF91CF9102
:1007600008958091F402E82FF0E0EB50FD4F99815D
:1007700090838F5F8093F4028093F30281E090E096
:10078000ECCF61E0CE0101960E944604F7CFCF92F4
:10079000DF92EF92FF920F931F93CF93DF937C0131
:1007A000CB018A012091F202222389F0EB016B0137
:1007B000C40ED51ECC15DD0569F06991D701ED9108
:1007C000FC910190F081E02DC7010995F3CF642FD2
:1007D0000E944604C801DF91CF911F910F91FF90B5
:1007E000EF90DF90CF9008951092160310921503AA
:1007F0001092F4021092F3020E9424048CE893E019
:100800000E94720482E693E00C946D04CF93C62F8D
:100810000E94F4038C2FCF910C9442047093F10248
:100820006093F0020895E2EEF2E01382128288EE05
:1008300093E0A0E0B0E084839583A683B78383E14F
:1008400091E09183808308951092A40381E08093C6
:10085000A2031092A10361E082E10E94020961E01B
:1008600083E10E940209E9EBF0E080818E7F8083C2
:1008700080818D7F808380E28093B80085E48093BF
:10088000BC000895880F8093BA0008952091590301
:10089000260F3327331F21323105ECF42091A403B6
:1008A000FC0190E080E0243069F082E00895A0919E
:1008B00059032191AC01455A5C4FA40FB52FB11DCE
:1008C0002C930196861798F380915903680F6093D3
:1008D000590380E0089581E0089590939E038093EA
:1008E0009D0308959093A00380939F03089585ED41
:1008F0008093BC008091BC0084FDFCCF1092A403C7
:10090000089585EC8093BC001092A40308951F9273
:100910000F920FB60F9211242F933F934F935F9333
:100920006F937F938F939F93AF93BF93EF93FF93B7
:100930008091B900887F803609F44CC008F03FC030
:10094000883209F4A8C018F5803109F49CC0B8F4C5
:10095000882309F4F9C0883009F495C0FF91EF911C
:10096000BF91AF919F918F917F916F915F914F91C7
:100970003F912F910F900FBE0F901F9018958831C7
:1009800009F489C0803251F78093370315C0803451
:1009900009F49EC048F48033B9F38833F9F68093A4
:1009A00037030E948104DACF803509F485C0883589
:1009B00009F496C0883491F60E947704CFCF883925
:1009C00009F48CC038F5883729F050F4883611F0D6
:1009D000803721F683E08093A4031092380357C038
:1009E000883809F47BC0803919F0803809F0B6CF17
:1009F00080913803803208F071C0E091380381E0C3
:100A00008E0F809338038091BB00F0E0E75CFC4FD1
:100A100080833DC0803B39F0E0F4803A09F479C02E
:100A2000883A09F09BCF84E08093A40310925A0384
:100A300010925903E0919F03F091A00309958091D2
:100A4000590381110FC081E08093590310925B0319
:100A500009C0803C09F476C0883C09F473C0883B27
:100A600009F07CCFE0915A0381E08E0F80935A0306
:100A7000F0E0E55AFC4F80818093BB0090915A03CF
:100A80008091590329C08091A3038093BB0085EC1A
:100A90008093BC0063CF90917C0380917B03981777
:100AA00058F5E0917C0381E08E0F80937C03F0E0A9
:100AB000E358FC4F8081E9CFE0917C0381E08E0F09
:100AC00080937C038091BB00F0E0E358FC4F80836F
:100AD00090917C0380917B039817C8F285E8D8CF6A
:100AE000E0917C0381E08E0F80937C038091BB00BA
:100AF000F0E0E358FC4F80838091A20381115CCF2A
:100B000081E08093A10384EA8093BC001092A40347
:100B100025CF0E94810480913803803230F4E09127
:100B20003803F0E0E75CFC4F10826091380370E01E
:100B3000E0919D03F0919E0389E393E00995109263
:100B400038030CCF85ECE0CF1092370335CF0F93ED
:100B50001F93CF93DF93EC01162F042F81E090E0D9
:100B60009983888386E391E09F838E8380EF9AEB5D
:100B7000A4E0B0E088879987AA87BB8780E29EE4DB
:100B8000A0E0B0E08C879D87AE87BF87673120F0FB
:100B90008FEF9FEF99838883073120F08FEF9FEFCE
:100BA0009983888361E0812F0E94C60860E0802FCE
:100BB0000E94C60860E0812F0E940209812F90E008
:100BC000FC01E158FF4FE491E88FFC01EA56FF4F2A
:100BD000E491F0E0EE0FFF1FE355FF4F85919491F4
:100BE0009A8F898F10E0F801E158FF4FE491EB8F65
:100BF000F801EA56FF4FE491F0E0EE0FFF1FE355D6
:100C0000FF4F859194919D8F8C8F8FEF9FEFAFEF6A
:100C1000BFE08A839B83AC83BD830E94A307688B5C
:100C2000798B8A8B9B8BDF91CF911F910F910895C8
:100C3000CF93DF93EC01F894E98DFA8D9281888D42
:100C4000809589238283EC8DFD8D91818B8D80959C
:100C500089238183EC8DFD8D92818B8D80958923F5
:100C60008283EC8DFD8D81819B8D892B8183EC8D21
:100C7000FD8D92818B8D8095892382838AE090E01F
:100C80000E940D08EC8DFD8D91818B8D80958923BF
:100C90008183EC8DFD8D92818B8D8095892382835C
:100CA000E98DFA8D8281988D892B82837894EC8DE1
:100CB000FD8D3B8D488559856A857B8520818C8992
:100CC0009D89AE89BF89232369F484179507A607F8
:100CD000B70740F40196A11DB11D8C8B9D8BAE8B87
:100CE000BF8BECCF481759076A077B0728F48EEFB4
:100CF0009FEFDF91CF910895F894EC8DFD8D828167
:100D00009B8D892B8283EC8DFD8D81819B8D892B21
:100D10008183EC8DFD8D82819B8D892B8283EC8D6F
:100D2000FD8D91818B8D809589238183EC8DFD8D47
:100D300092818B8D809589238283E98DFA8D9281B2
:100D4000888D8095892382837894EC8DFD8D3B8DF1
:100D5000488559856A857B8520818C899D89AE89E6
:100D6000BF89232349F484179507A607B70708F01E
:100D7000BECF81E090E0BDCF84179507A607B707E7
:100D800008F0B5CF0196A11DB11D8C8B9D8BAE8B4C
:100D9000BF8BE2CFCF92DF92EF92FF921F93CF9360
:100DA000DF93EC011C8A1D8A1E8A1F8A662309F4C0
:100DB00073C08881998197FD73C0162FF12CCE01E5
:100DC0000E94180697FD70C0F3941F11F8CF0E947F
:100DD000A307C888D988EA88FB886C197D098E0921
:100DE0009F09CC84DD84EE84FF84C616D706E8060E
:100DF000F90678F5CA80DB80EC80FD80C701B6017A
:100E00000E94A0092DEC3CEC4CEC5DE30E942E0A04
:100E10000E946A09AB01770F660B770B8C899D895D
:100E2000AE89BF898C199D09AE09BF098417950742
:100E3000A607B70770F48FEF9FEFAFEFBFE08A838D
:100E40009B83AC83BD830E94A307688B798B8A8BBD
:100E50009B8B8C899D89AE89BF89CA80DB80EC80A1
:100E6000FD808C159D05AE05BF0520F48A839B830C
:100E7000AC83BD83CA80DB80EC80FD80BC01CD01EA
:100E80006C197D098E099F09DF91CF911F91FF9009
:100E9000EF90DF90CF90089560E070E0CB01F4CF49
:100EA0006FEF7FEFCB01F0CF6EEF7FEF8FEF9FEF14
:100EB000EBCF1F920F920FB60F9211242F933F93F7
:100EC0008F939F93AF93BF938091AA039091AB03AD
:100ED000A091AC03B091AD033091A90326E0230F9C
:100EE0002D3768F129E8230F0396A11DB11D20932A
:100EF000A9038093AA039093AB03A093AC03B09390
:100F0000AD038091A5039091A603A091A703B09192
:100F1000A8030196A11DB11D8093A5039093A6037C
:100F2000A093A703B093A803BF91AF919F918F9116
:100F30003F912F910F900FBE0F901F901895029622
:100F4000A11DB11DD4CF2FB7F8946091AA03709161
:100F5000AB038091AC039091AD032FBF08953FB7D1
:100F6000F8948091A5039091A603A091A703B09156
:100F7000A80326B5A89B05C02F3F19F00196A11D17
:100F8000B11D3FBFBA2FA92F982F8827BC01CD01D3
:100F9000620F711D811D911D43E0660F771F881F31
:100FA000991F4A95D1F708958F929F92AF92BF9261
:100FB000CF92DF92EF92FF926B017C010E94AF070C
:100FC0004B015C01C114D104E104F104E9F00E9479
:100FD00069090E94AF07681979098A099B09683E67
:100FE00073408105910570F321E0C21AD108E10830
:100FF000F10888EE880E83E0981EA11CB11CC11474
:10100000D104E104F10429F7FF90EF90DF90CF9035
:10101000BF90AF909F908F900895000000008330A4
:10102000910528F0880F991F05970197F1F708950A
:10103000789484B5836084BD85B5836085BDEEE614
:10104000F0E0808181608083E1E8F0E082E08083ED
:10105000808181608083E0E8F0E08081816080832E
:10106000E1EBF0E0808184608083E0EBF0E0808160
:101070008160808386E880937A001092C100089591
:101080001F93CF93DF93182FEB0161E00E94C608F6
:10109000209739F460E0812FDF91CF911F910C945C
:1010A0000209CF3FD10511F461E0F5CFE12FF0E067
:1010B000E859FF4FE491E43031F140F4E230B1F00F
:1010C000E330E1F0C038D1057CF7E4CFE83029F116
:1010D000E93059F1E530B1F780918000806280936A
:1010E0008000D0938B00C0938A0004C084B58068D0
:1010F00084BDC7BDDF91CF911F91089584B58062F3
:1011000084BDC8BDF7CF8091800080688093800047
:10111000D0938900C0938800EDCF8091B0008068A3
:101120008093B000C093B300E5CF8091B00080629F
:101130008093B000C093B400DDCF843081F028F4F8
:101140008230E9F08330F9F00895883071F0893009
:1011500091F08530B9F4809180008F7D03C080913B
:1011600080008F778093800008958091B0008F7702
:101170008093B00008958091B0008F7DF9CF84B541
:101180008F7784BD089584B58F7DFBCFCF93DF9398
:1011900090E0FC01E158FF4F24918A569F4FFC01DB
:1011A00084918823C9F090E0880F991FFC01EF53C8
:1011B000FF4FA591B491FC01E954FF4FC591D49123
:1011C00061110DC09FB7F8948C91209582238C9368
:1011D0008881282328839FBFDF91CF9108956230B3
:1011E00051F49FB7F8943C91822F809583238C9380
:1011F000E8812E2BEFCF8FB7F894EC912E2B2C9308
:101200008FBFEACF1F93CF93DF93282F30E0F901F0
:10121000E859FF4F8491F901E158FF4FD491F9014A
:10122000EA56FF4FC491CC23A9F0162F81110E94DA
:101230009D08EC2FF0E0EE0FFF1FE954FF4FA59142
:10124000B4918FB7F894EC91111108C0D095DE23BA
:10125000DC938FBFDF91CF911F910895DE2BF8CFE4
:10126000CF93DF93282F30E0F901E859FF4F8491A5
:10127000F901E158FF4FD491F901EA56FF4FC491AB
:10128000CC23A1F081110E949D08EC2FF0E0EE0F1D
:10129000FF1FE355FF4FA591B491EC91ED2381E041
:1012A00090E009F480E0DF91CF91089580E090E034
:1012B000FACF08950E9418080E9459090E949200CE
:1012C000C0E0D0E00E94B2022097E1F30E9400004B
:1012D000F9CF08950E9471096894B1110C94280AFD
:1012E00008950E940D0A88F09F5798F0B92F99270A
:1012F000B751B0F0E1F0660F771F881F991F1AF001
:10130000BA95C9F714C0B13091F00E94270AB1E034
:1013100008950C94270A672F782F8827B85F39F033
:10132000B93FCCF3869577956795B395D9F73EF499
:1013300090958095709561957F4F8F4F9F4F089541
:10134000E89409C097FB3EF490958095709561955F
:101350007F4F8F4F9F4F9923A9F0F92F96E9BB2715
:101360009395F695879577956795B795F111F8CF91
:10137000FAF4BB0F11F460FF1BC06F5F7F4F8F4FFC
:101380009F4F16C0882311F096E911C0772321F0F2
:101390009EE8872F762F05C0662371F096E8862F8A
:1013A00070E060E02AF09A95660F771F881FDAF7E1
:1013B000880F9695879597F9089597F99F6780E824
:1013C00070E060E008959FEF80EC089500240A9497
:1013D0001616170618060906089500240A94121610
:1013E0001306140605060895092E0394000C11F443
:1013F000882352F0BB0F40F4BF2B11F460FF04C0F0
:101400006F5F7F4F8F4F9F4F089557FD9058440F48
:10141000551F59F05F3F71F04795880F97FB991F53
:1014200061F09F3F79F08795089512161306140610
:10143000551FF2CF4695F1DF08C01616170618069D
:10144000991FF1CF86957105610508940895E89478
:10145000BB2766277727CB0197F908950E94410A99
:101460000C94F4090E94E60938F00E94ED0920F07E
:10147000952311F00C94DD090C94E30911240C94CC
:10148000280A0E94050A70F3959FC1F3950F50E05A
:10149000551F629FF001729FBB27F00DB11D639F26
:1014A000AA27F00DB11DAA1F649F6627B00DA11DCC
:1014B000661F829F2227B00DA11D621F739FB00D72
:1014C000A11D621F839FA00D611D221F749F3327E2
:1014D000A00D611D231F849F600D211D822F762F7B
:1014E0006A2F11249F5750409AF0F1F088234AF058
:1014F000EE0FFF1FBB1F661F771F881F91505040C4
:10150000A9F79E3F510580F00C94DD090C94280A40
:101510005F3FE4F3983ED4F3869577956795B7954A
:10152000F795E7959F5FC1F7FE2B880F911D969564
:10153000879597F90895EE0FFF1F0590F491E02D20
:061540000994F894FFCFAE
:101546000101011415060708010203040506070038
:101556000000009803C7033503610338033F0352B5
:02156600030080
:00000001FF
